:100000000C943C010C945B010C945B010C945B011F
:100010000C945B010C945B010C945B010C945B01F0
:100020000C945B010C945B010C94FB180C94D1199B
:100030000C944B140C945B010C945B010C945B01CD
:100040000C945B010C945B010C945B010C945B01C0
:100050000C945B010C94D3140C945B010C945B0125
:100060000C945B010C945B010C945B010C945B01A0
:100070000C945B010C945B010C945B010C945B0190
:100080000C945B010C945B010C945B010C945B0180
:100090000C945B010C945B016E036E039A039A034C
:1000A0000F050F050F050F0502049B04AC04AC04FB
:1000B000421A691A611B691A611BB51AD81A611BA9
:1000C0002F1B3E1B00000000290064003D000A00B9
:1000D0003E000B003F00000034000000620063009F
:1000E0005200E2000000E1002B0039003C00170044
:1000F0002A001C00300040002F005C005D005E0004
:1001000000000000E000000035003A003B00220043
:10011000420023002E0041002D004C0049004B00FE
:100120004A000000000000001E001F002000210007
:1001300043002400250026002700440045004E000F
:100140004D0046000000000014001A0008001500D1
:10015000000018000C00120013005F006000610036
:1001600057004700000000000400160007000900C7
:1001700031000D000E000F00330059005A005B00E3
:1001800058000000E400E5001D001B0006001900F7
:10019000280010003600370032005300540055008C
:1001A0004800000000000000000000000000050002
:1001B0002C00110000000000380051004F005600D4
:1001C0005000E6002803490042004D0020004D0089
:1001D0006F00640065006C0020004D0020003100BD
:1001E000300031002F0031003000320000001003D9
:1001F00069007700300072006D003300720000006B
:100200000403090409022200010100A0FA09040004
:100210000001030101000921110100012240000732
:100220000581030800011201000200000008EDFE34
:10023000000001000102000105010906A1010507F6
:1002400019E029E71500250195087501810295013E
:10025000750881010507190029FF150026FF009583
:100260000675088100050819012905950575019194
:1002700002950175039101C011241FBECFEFD0E29A
:10028000DEBFCDBF11E0A0E0B1E0EEEDF7E300E0AE
:100290000BBF02C007900D92AA32B107D9F722E036
:1002A000AAE2B1E001C01D92A733B207E1F70E94B4
:1002B0002B110C94ED1B0C940000249A259A269A7D
:1002C0002C9A2D9A2E9A089580FF02C02C9801C076
:1002D0002C9A81FF02C02E9801C02E9A82FF02C084
:1002E0002D9801C02D9A0C94350281E0089581E08B
:1002F00008950C94770108950C947B011F93CF937C
:10030000DF9300D000D01F92CDB7DEB749835A8368
:100310006B8330912D0189819A81311114C066233C
:1003200059F0222349F00E944007182F682F898135
:100330009A810E94E90603C00E941407182F698160
:100340007A81812F04C00E94400769817A810F90D1
:100350000F900F900F900F90DF91CF911F910C9401
:10036000920EFC01262F408151816281738184812C
:100370000C947E0181E00895CF93DF93EC0160E05F
:100380000E94B101BE01DF91CF910C947C010C94CD
:10039000C30F0C94BF0F08950E9493050E94CB01D8
:1003A0002FEF84E39CE0215080409040E1F700C0B3
:1003B00000000C94F9140F931F93CF93DF938C01DB
:1003C00061E00E94B101EC01B8010E94790188232B
:1003D000F1F1B801CE010E9424138823C1F1B801C4
:1003E000CE010E943811882391F1B801CE010E94FC
:1003F0008012882361F1F8018281882309F1CB35CD
:100400008DE5D807C1F050F4C115FCE5DF0781F098
:10041000CF3DDC45A9F40E94710C19C0CC35EDE547
:10042000DE0761F0CD35DD4559F40E94BA0B08C0F6
:100430000E94CC010CC00E94C30B02C00E94C60BDC
:10044000C801DF91CF911F910F910C94750180E04D
:10045000DF91CF911F910F9108950E942D140C945C
:1004600044020E9447020C943314089581E00895D9
:100470000C9436020895CF93C82F0E9464018C2FEC
:100480000E943802CF91089580E00C943B020E94B4
:1004900080130C943B020E94801390912C018917C9
:1004A00021F080932C010C943B020895CF93DF93AD
:1004B000CDB7DEB72B970FB6F894DEBF0FBECDBF1A
:1004C0004F83588769877A878B8761110E94060B53
:1004D0009E012F5F3F4F86E0F90111928A95E9F75F
:1004E00085E0FE013796D90101900D928A95E1F7DA
:1004F00089819A814C815D81452B31F09F3F31F498
:1005000091E08F3F19F403C091E001C090E090FFAB
:1005100009C049815A816B817C818D819E810E94B5
:10052000270A05C0C9010E94BA018111F2CF2B969A
:100530000FB6F894DEBF0FBECDBFDF91CF91089507
:10054000FC01808191810E9482070895CF938823C6
:1005500071F1C82F8CEF8C0F813AD0F46C2F809101
:100560000201909103010E94CF13882349F06C2F60
:1005700080910201909103010E9407140E94280BB0
:100580006C2F80910201909103010E9405140CC010
:1005900080E28C0F883058F4C77081E001C0880F6A
:1005A000CA95EAF70E94E90ACF910C94280BCF91E3
:1005B0000895882349F1682F8CEF860F813A38F42B
:1005C00080910201909103010E9407140CC080E207
:1005D000860F883050F4677081E001C0880F6A95FB
:1005E000EAF70E94EF0A0C94280B8BE5860F833004
:1005F00020F480E090E00C949713685A673120F45F
:1006000080E090E00C94AD1308951F93CF93DF9397
:10061000182FEB010E94A602209741F08FE99FE07E
:100620000197F1F700C000002197F6CF812FDF91ED
:10063000CF911F910C94D902893319F060E070E0DA
:1006400002C060E570E00C940503882321F00E944D
:10065000E90A0C94280B0895882321F00E94EF0AE0
:100660000C94280B0895CF92DF92EF92FF920F9394
:100670001F93CF93DF937C01D62FC72FFC011281EC
:10068000058102950F700E94DF0A8823B9F01123BB
:10069000A9F08C2F807F803421F080E28D0F88308C
:1006A00068F08091050282FD09C082E00E94880BFB
:1006B0000E94DF0A91E0D82ED92601C0D12CCC2E81
:1006C000C2948FE0C8228C2D90E08C30910508F008
:1006D000A6C1FC01E45BFF4F0C94951B8C2F807F1F
:1006E000CF70882311F0C295C07F112399F0CC23DD
:1006F00009F481C180E28D0F883010F0D11104C05F
:100700008C2F0E94E90A03C08C2F0E94F90A0E94D4
:10071000280B71C18D2F0E94D902CC2309F47FC10F
:1007200080E28D0F883038F1DD2329F18C2F0E9473
:10073000FF0A24C08C2F807FCF70803211F0C295C9
:10074000C07FDD2319F0D130A1F13DC080910502B9
:1007500082FF17C0112349F0CC2329F08C2F0E946F
:10076000E90A0E94280B80E047C180E00E94D9027C
:10077000CC2309F454C18C2F0E94EF0A0E94280B4D
:100780004EC1112371F0002341F0013031F40E9479
:10079000090B8C2B0E94110B42C10E94090B8C2B60
:1007A0001DC0002319F0013009F439C10E941E0B4D
:1007B00025C0112321F0063008F031C10EC00530EC
:1007C00008F02DC11BC0112361F0002331F0F701A7
:1007D000858180FF10C18F7085838C2F0E94250337
:1007E0001EC1002359F0D93309F016C1FFEF07EEFF
:1007F00013E0F15000401040E1F70CC18C2F0E9433
:100800002C030DC18C2F837009F047C011110BC14F
:100810002D2F229526952770220F220F6D2F6F7096
:10082000862F90E0A0E0B0E0022E04C0880F991F50
:10083000AA1FBB1F0A94D2F7D4FF10C04FE050E0AC
:1008400060E070E004C0440F551F661F771F2A95B3
:10085000D2F7409550956095709503C040E050E008
:10086000BA01C695C695C3708A019B01082B192B46
:100870002A2B3B2BC901B801C23049F058F4C130D2
:1008800019F00E94FF05CFC00E94ED05CCC00E9468
:100890001106C9C00E94EB05C6C0112319F08C2FA8
:1008A000817001C08695882309F4BDC02D2F229543
:1008B00026952770220F220F6D2F6F70862F90E0E4
:1008C000A0E0B0E0022E04C0880F991FAA1FBB1F32
:1008D0000A94D2F7D4FF10C04FE050E060E070E01F
:1008E00004C0440F551F661F771F2A95D2F7409505
:1008F00050956095709503C040E050E0BA01C695F0
:10090000C695C3708A019B01082B192B2A2B3B2B00
:10091000C901B801C23049F058F4C13019F00E9441
:10092000C40681C00E94B2067EC00E94D6067BC06B
:100930000E94250678C0CF70112339F08C2F0E94B9
:100940004B068D2F0E9425036EC08D2F0E942C0315
:100950008C2F0E946C0667C0D23F21F128F4D03F53
:1009600041F0D13FC1F043C0D33F19F1D43F79F0FA
:100970003EC0112341F0053008F051C08C2F8F711B
:100980000E9491064CC0063008F049C0F7CF809114
:10099000050282FF18C0112339F08C2F8F710E943D
:1009A0004B063DC01123C9F38C2F8F710E946C063A
:1009B00036C0112329F08C2F8F710E9436062FC06C
:1009C0000E9431062CC0112349F0CF718C2F0E9458
:1009D0004B0663E08C2F0E946D0B21C081E00E94CA
:1009E000880B0230E0F082E00E94880B18C01123CF
:1009F00031F0002391F28D2F0E94A60210C0002337
:100A000099F2D93349F41FEF27EE33E0115020401B
:100A10003040E1F700C000008D2F0E94D90288EF1E
:100A20008C0D843020F40E9480130E943B02DD2054
:100A3000C9F00E94DB0A80FD15C0F70112820E94F6
:100A4000D50A0E944B06C7010E9453050E94D50A91
:100A5000DF91CF911F910F91FF90EF90DF90CF909A
:100A60000C946C06DF91CF911F910F91FF90EF9046
:100A7000DF90CF9008950F931F93CF93DF93EC01F6
:100A8000688179818A810E948D078C010E94E80625
:100A90000E94D905B801CE010E943303DF91CF91A6
:100AA0001F910F910895CF93DF93EC019881898175
:100AB0002B813C81232B31F08F3F31F481E09F3F2C
:100AC00019F403C081E001C080E080FD1DC0CE01AB
:100AD0000E94DB01811110C00E94DF0A8823A1F06F
:100AE0008A81882389F08091050282FD0DC082E011
:100AF000DF91CF910C94880BCE010E943B05CE0173
:100B0000DF91CF910C94BC01DF91CF9108950E94A9
:100B1000060B0C94280B80910201909103010E9416
:100B200009140C9487050E94F60A0C948B05929583
:100B30009F70963079F010F4925001C09A50923024
:100B400068F4803F69F018F4883E40F409C0843F9F
:100B500029F406C0883E20F0813F11F080E008951E
:100B600081E00895FC01808191810E9482070E94AA
:100B700097050895CF93DF9300D000D01F92CDB793
:100B8000DEB70F900F900F900F900F90DF91CF91E5
:100B90000895CF93DF9300D000D000D0CDB7DEB75B
:100BA00026960FB6F894DEBF0FBECDBFDF91CF9172
:100BB0000895089508950C94DA050C94DB050E94BD
:100BC000DD0560938201709383018093840190938B
:100BD00085010C9487050C94DF050F931F930091FA
:100BE0008201109183012091840130918501602B55
:100BF000712B822B932B1F910F910C94DF050F9378
:100C00001F93009182011091830120918401309102
:100C1000850160237123822393231F910F910C94EC
:100C2000DF050F931F9300918201109183012091A2
:100C300084013091850160277127822793271F91B6
:100C40000F910C94DF050C94DA050E942306609343
:100C50007E0170937F0180938001909381010C94B9
:100C6000870560E070E0CB010C9425060F931F937D
:100C700041E050E060E070E08A019B0104C0000F99
:100C8000111F221F331F8A95D2F7C901B8011F9186
:100C90000F910C9425060F931F9341E050E060E004
:100CA00070E004C0440F551F661F771F8A95D2F766
:100CB00080917E0190917F01A0918001B09181018E
:100CC0008A019B01082B192B2A2B3B2BC901B80148
:100CD0001F910F910C9425060F931F9341E050E054
:100CE00060E070E004C0440F551F661F771F8A95AF
:100CF000D2F7409550956095709580917E019091C6
:100D00007F01A0918001B09181018A019B0108239C
:100D100019232A233B23C901B8011F910F910C9479
:100D200025060F931F9341E050E060E070E004C09F
:100D3000440F551F661F771F8A95D2F780917E0159
:100D400090917F01A0918001B09181018A019B0166
:100D5000082719272A273B27C901B8011F910F919E
:100D60000C9425060F931F9300917E0110917F0133
:100D70002091800130918101602B712B822B932B6C
:100D80001F910F910C9425060F931F9300917E01E4
:100D900010917F01209180013091810160237123A6
:100DA000822393231F910F910C9425060F931F9379
:100DB00000917E0110917F0120918001309181018D
:100DC00060277127822793271F910F910C94250686
:100DD000089520E1929F800D1124E82FE695E69575
:100DE000E695877051E001C0550F8A95EAF785E0D6
:100DF000E89FF0011124E25DFE4F20E030E070E05A
:100E00004081CB01022E02C0969587950A94E2F7A5
:100E10008170819584278523842781932F5F3F4F9D
:100E20002530310569F7089520E1929F800D112446
:100E3000682F669566956695982F977085E0689FF0
:100E4000B001112440E050E080E0FB01E40FF51F09
:100E5000E25DFE4F208130E0092E02C036952795D5
:100E60000A94E2F721703327042E01C0220F0A945E
:100E7000EAF7822B4F5F5F4F4530510531F70895F8
:100E8000BF92CF92DF92EF92FF920F931F93CF9377
:100E9000DF938C01C0907E01D0907F01E0908001B3
:100EA000F09081018091820190918301A091840151
:100EB000B0918501C82AD92AEA2AFB2ACFE1D0E0DD
:100EC000D701C6010C2E04C0B695A79597958795B6
:100ED0000A94D2F780FD04C0219790F7B12C07C087
:100EE000BC2EB8018C2F0E94A70E0197A9F38B2D61
:100EF000DF91CF911F910F91FF90EF90DF90CF90F6
:100F0000BF900895CF93DF93EC010E944007BE018C
:100F10000E94A70EDF91CF9108951F93CF93DF9387
:100F2000EB0190912D01992321F0CB010E948207C2
:100F300013C0882349F0CB010E944007182F682F67
:100F4000CE010E94E90604C0CB010E941407182FAD
:100F5000BE01812F0E94A70EDF91CF911F910895AE
:100F60001F93CF93DF93C091860116E08091870194
:100F7000C81799F0D0E01C9FF0011D9FF00D1124BF
:100F8000E857FE4F40815181628173818481958150
:100F90000E94C9052196C770E9CFDF91CF911F91BB
:100FA00008954091B8015091B9016091BA017091D2
:100FB000BB018091BC019091BD010C94C905EF92D9
:100FC000FF920F931F93CF93DF938091BD01829582
:100FD0008F7009F065C08091BA01882309F460C060
:100FE00080918601F09087011091B8010091B901BC
:100FF0006091BB017091BC0191E01F3F09F090E04E
:10100000C0910001D0910101292F96E0E92E8F15A2
:1010100009F446C06115710521F00F3F21F030E061
:1010200003C031E001C0322F90E030FD36C0E89EB1
:10103000F001E99EF00D1124DF01A857BE4F119673
:101040003C911197301329C03C91311326C0129660
:101050003C911297311121C013964D915C911497D8
:10106000461B570B4C175D07C0F48091BD018F7074
:1010700080618093BD01E357FE4F80818F70806156
:10108000808388EB91E00E945305DF91CF911F91FF
:101090000F91FF90EF900C94B00701968770B7CF37
:1010A000DF91CF911F910F91FF90EF9008959F9244
:1010B000AF92BF92CF92DF92EF92FF920F931F9366
:1010C000CF93DF93CDB7DEB761970FB6F894DEBF4D
:1010D0000FBECDBF8C0185E0F801DE011D960190A9
:1010E0000D928A95E1F7D8011296EC909091B80193
:1010F000E091B9012091BB013091BC01211531056E
:1011000031F0EF3F31F481E09F3F19F403C081E0FB
:1011100001C080E0B82FB1709B2E80FD47C1D8017F
:101120004C9111965C9111971396AD90BC901497C9
:1011300088EBC82E81E0D82EF090BA01B501621B71
:10114000730B2091000130910101FF2009F4D9C0F7
:101150008091BD016217730708F095C0282F207F8A
:1011600009F052C05E1313C0491311C0FE2CE110E8
:101170000EC08F7080618093BD010E94D107C601AF
:101180000E9453058091BD01F80185834DC1AB28B4
:1011900031F05F3F31F481E04F3F19F403C081E04B
:1011A00001C080E080FD03C081E08E2502C080E0A8
:1011B00090E0F82FF170FF2E80FF1CC08091860117
:1011C0002091870136E0821709F40BC190E0389F27
:1011D000F001399FF00D1124E857FE4F618156133D
:1011E00006C06081461303C06281E61203C0019607
:1011F0008770E9CFFE2CEE2009F416C18091BD0165
:1012000081608093BD0154C05E1306C0491304C0C1
:10121000E11002C0F80199C0C8010E94B2058823FC
:1012200061F1EE2051F12091BD01822F82958F70E6
:1012300090E0029774F08091B8019091B90198877D
:101240008F831986BB86AA862C87CE0107960E94BB
:10125000530586E0F801A8EBB1E001900D928A9564
:10126000E1F70E94DF070E94D1070AC05E1711F163
:10127000C8010E94B20581112CC0C8010E9453050B
:10128000FF24F394D1C0282F207F81F77A2DB98ACB
:10129000A88A6E2D89890E94BA0588EB91E00E9488
:1012A000530586E0D6011D928A95E9F70E94D10781
:1012B000F12CBAC04913DCCFE110DACFF8018583F5
:1012C000C8010E94530586E0D6011D928A95E9F770
:1012D000ABC0EE2091F22091BD01822F82958F70DC
:1012E00090E002970CF4B5CF8091B8019091B901CC
:1012F0009A8389831B82BD82AC822E83CE010196A4
:10130000A6CF6217730708F044C0FE2CEE2009F444
:10131000B4CF5E1330C049132EC02091BD0120FD13
:1013200021C0822F82958F70482F50E041155105C2
:10133000C9F0F80125834F30510541F08F5F982F98
:101340009295907F822F8F70892B8583C8010E9490
:10135000530586E0F801A8EBB1E001900D928A9563
:10136000E1F73CC086E0F801A8EBB1E001900D92F6
:101370008A95E1F759C0C8010E94B205811169CF71
:101380008091BD0181608093BD01C8010E94530519
:101390004BC07A2DB98AA88A6E2D89890E94BA0518
:1013A00086E0D6011D928A95E9F718C0EE2009F46F
:1013B00064CFC8010E94B205F82E882309F45DCFDE
:1013C00086E0F801A8EBB1E001900D928A95E1F773
:1013D00088EB91E00E94A0020E94DF070E94D107E3
:1013E00023C04D875E878D859E850E948207292FA9
:1013F00022952F70223028F49F7039F0811105C09A
:101400000BC0243028F49F7049F4805E883020F0AF
:10141000C8010E9453059F2CF92C06C0D8011596CF
:101420009C91907F91F7F8CF8F2D61960FB6F8942D
:10143000DEBF0FBECDBFDF91CF911F910F91FF9007
:10144000EF90DF90CF90BF90AF909F9008951F9343
:10145000CF93DF93CDB7DEB72C970FB6F894DEBFEE
:101460000FBECDBF4F83588769877A878B879C874C
:10147000CE0107960E9457088823D1F09F81888566
:101480002A853B85232B31F08F3F31F481E09F3F4C
:1014900019F403C081E001C080E080FD47C04F81A6
:1014A000588569857A858B859C850E94C9053EC0D3
:1014B00086E0FE013796DE01119601900D928A9525
:1014C000E1F7FF81E8856A857B856115710531F05B
:1014D000EF3F31F481E0FF3F19F403C081E001C028
:1014E00080E080FD23C02091870130E0C901019692
:1014F000877099274091860150E084179507F1F194
:10150000F983EA837D836C8396E0929FD001939F59
:10151000B00D1124A857BE4FFE01319601900D92D7
:101520009A95E1F7809387010E94B00716E08091B9
:10153000860190918701891771F1189FC0011124CC
:1015400088579E4F0E945708882329F1E091860111
:101550001E9FF0011124E857FE4F408151816281A6
:101560007381848195810E94C9058091860190E0F4
:1015700001968770992780938601D9CF0E949305A1
:101580001092870110928601E8EBF1E086E0DF011E
:101590001D928A95E9F72C960FB6F894DEBF0FBE20
:1015A000CDBFDF91CF911F9108958091C6018595A0
:1015B0008595859508958091C601877008959091CD
:1015C000C601977081E009F480E008958091D1010F
:1015D00008959091D101892B8093D1010895809530
:1015E0009091D10189238093D10108951092D10166
:1015F00008959091D001892B8093D0010895809512
:101600009091D00189238093D00108951092D00148
:1016100008958091C701089508950C940C0B0C94C3
:101620000D0B9091050292FD08C09091C70198178B
:1016300021F08093C7010C940F0B08958091C7018E
:10164000882329F01092C70180E00C940F0B0895B5
:10165000CF93DF93E0910201F09103018091D101DA
:101660008083E0910201F091030190818091D0018B
:10167000892B80838091C701882381F0E09102014A
:10168000F09103019081892B8083809102019091D8
:1016900003010E94C31381110E941E0BC09102011D
:1016A000D091030148E050E06EEB71E0CE010E9462
:1016B0009E1B892B69F088E0FE01AEEBB1E0019042
:1016C0000D928A95E1F7CE01DF91CF910C948C13A6
:1016D000DF91CF9108950C940C0B9091050292FD2F
:1016E00010C098E0899F90011124262B2093C601F9
:1016F0000E944B068091C6018595859585950C9431
:101700006B0B0C944B061092C60180E00C946B0B93
:101710002091C601809582238093C601982F9770EF
:1017200099F430E0482F082E000C550B241735078C
:1017300059F09091050292FD07C085958595859594
:101740000E946C060C94830B08959091050292FB05
:10175000222720F9281769F080FB92F9909305025F
:1017600080910402909105020E94ED0B82E00C949E
:10177000880B08958091050282FB882780F991E00B
:1017800089270C94A50B81E00C94A50B80E00C94A8
:10179000A50B80E090E00E94B31B21E0893E9E4FA4
:1017A00009F020E0822F089582E090E00C94AB1BBA
:1017B00083E090E00C94AB1BCF9384E090E00E9418
:1017C000AB1BC82F82E290E00E94AB1B2C2F30E0B5
:1017D000A901582BCA01CF910895CF93C92F682F23
:1017E00084E090E00E94B91B6C2F82E290E0CF91E0
:1017F0000C94B91BAB01BC018FE090E00C94CB1BA7
:10180000AB01BC0183E190E00C94CB1B60E070E085
:10181000CB010C94000C60E070E0CB010E94FA0B4D
:101820000C94060C69EE7EEF80E090E00E94D71BDE
:1018300060E082E090E00E94B91B60E083E090E00D
:101840000E94B91B109282011092830110928401B0
:101850001092850160E084E090E00E94B91B60E096
:1018600082E290E00E94B91B60E085E090E00E9477
:10187000B91B60E086E090E00E94B91B6FEF87E043
:1018800090E00E94B91B40E050E0BA0188E090E08F
:101890000E94CB1B60E08DE090E00E94B91B40E00D
:1018A00050E0BA0188E190E00E94CB1B60E087E144
:1018B00090E00E94B91B40E050E0BA018CE190E05A
:1018C0000E94CB1B60E070E080E290E00E94D71B9A
:1018D00040E050E0BA0188E190E00E94CB1B0C94FC
:1018E0000B0C0C94120C682F8EE090E00C94B91B3A
:1018F000CF93DF9390E1899FD001112420E030E065
:1019000080E090E0C1E0D0E0F901EA0FFB1FEE0FAC
:10191000FF1FEC53FF4FE491EE2371F0AE01022E56
:1019200002C0440F551F0A94E2F7FA01E623F72399
:10193000EF2B11F0842B952B2F5F3F4F203131057A
:1019400019F7DF91CF9108950E94B8146093E601D2
:101950007093E7018093E8019093E9016093E201BD
:101960007093E3018093E4019093E501089585B7B6
:10197000806885BF85B7806885BF089581E0089538
:101980000C94BE0C08950C94C20C0C94C20C0C94D4
:10199000C50C0C94C20C0E94B70C83E89FE00E9417
:1019A00076130E94C90C0C945D010E94C30C0C9428
:1019B000C20C0E94860F0C943A020E94A3140E944B
:1019C0007A100E94D90C0C94C70C4F925F926F92C0
:1019D0007F928F929F92AF92BF92CF92DF92EF92BF
:1019E000FF920F931F93CF93DF93CDB7DEB72A9764
:1019F0000FB6F894DEBF0FBECDBF0E948F10582ED9
:101A000081110E94A40C32ED832E31E0932E00E070
:101A100010E0402E802F0E94AA0F6C01F401A190CB
:101A2000B1904F01A826B926A114B104B1F40F5FFB
:101A30001F4F0830110569F78FEF89838A831B8256
:101A40000E94AC148160782F9D838C8349815A81D8
:101A50006B818D810E94560240C0BC01802F0E9484
:101A6000780C3C01019786219721892BC9F0F12C34
:101A70004F1005C0F394F8E0FF12FACF11C08F2D7C
:101A80000E94AA0FBC018F2D0E94780C86219721FD
:101A90009C012150310982239323892B59F3C7CF0D
:101AA0008091EA0181FD0E94B30F712CEE24E39432
:101AB000F12CC5018E219F21892B51F10E94C00C70
:101AC000811110C0000F111FF801EE52FE4F8081EE
:101AD0009181E826F926F182E08281E051101FC051
:101AE00080E01DC07E824F82CE20DF2081E0CD28A5
:101AF00009F480E088870E94AC148160782F9A876F
:101B000089874E815F8168858A850E945602DACF77
:101B10007394EE0CFF1C80E17812CBCF88CF2A960D
:101B20000FB6F894DEBF0FBECDBFDF91CF911F91EE
:101B30000F91FF90EF90DF90CF90BF90AF909F906C
:101B40008F907F906F905F904F9008950E94E50C6A
:101B50000C944B02CF93DF930E94AC0EEC018115E5
:101B600023E59207A0F5811532E5930708F09EC0A2
:101B7000811540E29407C0F4811551E0950708F003
:101B8000CDC0853A910550F48430910508F0C6C067
:101B9000019709F0C0C081E090E0C1C0805E91096A
:101BA000089708F4BBC0B7C0C11581E5D80708F095
:101BB00077C0C11520E5D20708F051C0C11530E447
:101BC000D30708F4A8C0DF70CE01906AA8C08115C1
:101BD00046E5940700F5811555E5950708F081C0A5
:101BE000C11584E5D80708F076C0CE018370992727
:101BF00021E030E002C0220F331F8A95E2F79C2FCC
:101C00009695969540E2949FE0011124C22BD32B28
:101C1000CE019A6884C081152AE5920780F4811567
:101C200039E5930708F066C0811548E5940708F484
:101C300072C0D82FCC27CE01806F906A70C09056AA
:101C40008115904208F067C08D2F8F710E94400F60
:101C5000DD27D0628F71AE01582BCA0160C0CE0162
:101C600074E0969587957A95E1F7282F23703C2F9D
:101C7000337081E090E002C0880F991F3A95E2F737
:101C80009C68AC01522B9A019C2F9F70969596955B
:101C900050E2959FE0011124C9018C2B9D2B3FC080
:101CA000DC2FCC27CE01816F906A39C083709927D1
:101CB00021E030E002C0220F331F8A95E2F79C2F0B
:101CC0009695969580E2989FE0011124C22BD32B24
:101CD000CE019C6824C0DC2FCC27CE01846F906A93
:101CE0001EC00E94400F8F7190E0D82FCC27CE01EC
:101CF000906215C08F700E94400F94E0D695C795F2
:101D00009A95E1F7CF70D0E0DC2FCC27D0699E0107
:101D1000282BC90104C080E090E001C0CE01DF9112
:101D2000CF910895E72FF0E098E0899FE00DF11D35
:101D3000112484E0EE0FFF1F8A95E1F7E60FF11DF5
:101D4000EE0FFF1FEC53FF4F8591949108950E9471
:101D5000920E0E94AA0D08958238910569F1B0F49F
:101D60008133910509F46DC048F48932910509F475
:101D700063C08A32910509F469C0089585339105DD
:101D800009F455C089339105B9F00895833E910552
:101D900069F138F4803E9105B1F0823E910509F178
:101DA0000895863E9105A9F1873E9105B9F1843EDB
:101DB000910509F064C023C02091040220FD4FC0AA
:101DC00021FD4DC008958091040280FD44C08091A2
:101DD000050280FF44C08091040284FD42C083EE6E
:101DE0004DC08091040282FF38C0F5CF809104027B
:101DF00082FD33C08091050280FD31C0ECCF80911F
:101E0000050281FF32C08091040284FD2AC087EE62
:101E100035C08091040283FF26C0F5CF8091040273
:101E200083FD21C08091050281FD1FC0ECCF809110
:101E3000040285FD1CC01DC08091040285FD19C0EF
:101E400016C08091040286FD16C017C0809104025E
:101E500086FD13C010C089E311C082EE0FC080EE72
:101E60000DC080E00BC086EE09C084EE07C089E299
:101E700005C085E303C08AE201C081E390E00895D4
:101E80009091040292FF0DC0282F2871283019F478
:101E9000877F846006C0282F2471243011F48B7F43
:101EA000886093FF0DC0282F2871283119F4877E90
:101EB000846106C0282F2471243111F48B7E88613F
:101EC0002091050220FF0DC0382F3871383019F4E9
:101ED000877F816006C0382F3171313011F48E7FD9
:101EE000886021FF0DC0282F2871283119F4877EC2
:101EF000816106C0282F2171213111F48E7E886105
:101F000094FD877E089580E0089508950E94C90B8E
:101F1000811102C00E94710C0E94D40B8093EA01CF
:101F20000E94DC0B90930502809304020E94850FAF
:101F30000E94D80B682F70E080E090E00E94EB05D3
:101F400060917E0170917F0180918001909181016B
:101F50000C942306E82FF0E0EE0FFF1FEA5EFD4F22
:101F6000808191810895089580EA8A95F1F7089516
:101F700000C008950C94B40F08950C94BC0F0C94F9
:101F8000BD0F0C94BC0F0C94C10FF894E82FE29590
:101F9000EF70F0E031A1282F2F7081E090E001C0B8
:101FA000880F2A95EAF7982F9095932391A392A1F1
:101FB000892B82A3789408950F931F93CF93DF9377
:101FC000C1E1D1E089918F3F11F00E94C50F81E0FE
:101FD000C132D807B9F7C1E2D1E009E211E0899135
:101FE0008F3F11F00E94C50F0C171D07C1F7DF913D
:101FF000CF911F910F910895AF92BF92DF92EF9210
:10200000FF920F931F93CF93DF93C62FD0E0CF5E45
:10201000DE4F28812F3F09F463C08A01F62EE92E96
:10202000D82EF894E22FE295EF70F0E091A1822F84
:102030008F7021E030E001C0220F8A95EAF7892FE6
:10204000822B81A382A12095282322A378940E9429
:10205000B80F81E2A82E81E0B82EED2DFE2D9F0154
:10206000205F3F4FE12CA80140955095D5016D911F
:102070005D016F3FC9F0862F82958F7090E0DC0183
:1020800090968C9190E06F7002C0959587956A95B7
:10209000E2F780FD09C080819181802B912B918393
:1020A0008083EE24E39406C080819181842395236C
:1020B000918380833296E217F307C1F688818F3FC0
:1020C00011F00E94C50F6E2D8F2DDF91CF911F91C2
:1020D0000F91FF90EF90DF90BF90AF900C94BA0FEC
:1020E000DF91CF911F910F91FF90EF90DF90BF9004
:1020F000AF9008950E94DC0F80E1E6E1F2E0DF019D
:10210000982F1D929A95E9F7E6E0F2E0DF011D9223
:102110008A95E9F788E00E94E4100C94C701CF92F9
:10212000DF92FF920F931F93CF93DF93CDB7DEB76C
:1021300060970FB6F894DEBF0FBECDBF8E010F5F64
:102140001F4F80E1F80111928A95E9F7F12CCC2418
:10215000C394D12CA6016F2DC8010E94FC0FF394EB
:10216000CC0CDD1CF0E1FF12F5CF40E150E0B801EE
:1021700086E092E00E949E1BFF24F394009709F4EE
:10218000F12C892B41F080E1F801A6E0B2E001904A
:102190000D928A95E1F72F2D48E066E172E086E026
:1021A00092E00E94E5100E94C9018F2D60960FB643
:1021B000F894DEBF0FBECDBFDF91CF911F910F917D
:1021C000FF90DF90CF9008950895FF920F931F9393
:1021D000CF93DF93F82E092F162FD72FC42F22234A
:1021E00049F081E08093ED010E94AC149093EC01E2
:1021F0008093EB018091ED018823D9F08091EB0170
:102200009091EC010E94C414059798F0EF2DF02FE7
:10221000A12FBD2F80E090E04C2F50E08417950750
:1022200034F4219131912D933D930196F7CF109283
:10223000ED01DF91CF911F910F91FF9008950E94C2
:1022400067160E94DD0C0C9473160E9477160E948C
:10225000A60D0C9491160E944A140E944E160E94DC
:10226000CB0C0E941F110E9425110E94D50CFBCFA0
:10227000CF93DF93EC01FB018281882309F43CC1F9
:10228000C430FDE5DF0760F4CB3F9CE5D90788F457
:102290009E0122503C452431310508F02EC109C071
:1022A000C236EDE5DE0729F0C63AFDE5DF0709F0A5
:1022B00024C10E94DC0B9093050280930402C1317B
:1022C0008CE5D80709F4C6C008F042C0C930ECE577
:1022D000DE0709F49BC000F5C5308CE5D80709F48A
:1022E00085C078F4C330ECE5DE0709F478C008F067
:1022F0007AC0C230DC4509F0F5C0809104028160EB
:10230000EFC0C7309CE5D90709F478C008F07AC05F
:10231000809104028061E4C0CD30FCE5DF0709F460
:1023200087C058F4CB309CE5D90709F479C008F090
:102330007BC08091040288606FC0CF30FCE5DF076E
:1023400009F480C008F082C080910402877FC8C071
:10235000CE3F9CE5D90709F471C000F5C531FCE515
:10236000DF0709F485C068F4C3319CE5D90709F497
:1023700075C008F095C00E949305809104028F7784
:10238000AFC0CC3FFCE5DF07A9F108F054C0CB3F5C
:10239000DC4509F0A7C08091050240C0C230EDE5E0
:1023A000DE0709F489C058F4C1158DE5D80709F492
:1023B0005AC008F069C08091050282602FC0C23601
:1023C000EDE5DE0709F47CC0C63AFDE5DF0709F458
:1023D00081C0C330DD4509F085C080E06EC08091CA
:1023E000040282607DC08091040216C080910402C4
:1023F000886076C08091050282604FC0809104029F
:1024000080626EC08091040280646AC00E9493055D
:1024100080910402806864C0846062C081603DC0B5
:10242000809104028E7F5CC0809104028D7F58C031
:102430008091040216C08091050218C080910502A7
:102440008D7F2BC0809104028F7E4AC08091040250
:102450008F7D46C0809104028F7B42C08091040230
:10246000877F8B7F3DC0809105028D7F8E7F15C059
:102470008091040282FB222720F991E0922790FBB1
:1024800082F990FB83F92CC080910502982F9095DA
:1024900091708E7F892B90FB81F98093050222C079
:1024A0000E9493058091040287FB222720F991E086
:1024B000922790FB87F914C081E00E94730C12C030
:1024C0008091040284FB222720F991E0922790FB5F
:1024D00084F906C080910402982F909590FB80F9B2
:1024E0008093040280910402909105020E94ED0BFA
:1024F0000E94930580E001C081E0DF91CF910895B3
:10250000CF93DF9386319C4541F5EB010E94E60AAB
:10251000982F8A812091020130910301882379F05C
:102520009A7A81E009F480E08093EE01911102C073
:1025300069E201C065E3C9010E9405140AC08091E7
:10254000EE01811102C069E201C065E3C9010E9488
:1025500007140E94280B80E001C081E0DF91CF9139
:1025600008950F931F93CF93DF93C42FD22FFC01B5
:1025700082818823C9F04093F1010E94AC149093AA
:10258000F0018093EF0180E28C0F883008F057C093
:10259000C77081E001C0880FCA95EAF7DF91CF913B
:1025A0001F910F910C9425038091F101481330C0C5
:1025B0008091EF019091F0010E94C414883C910534
:1025C00038F510E21D0FCD17B9F080E28C0F88307E
:1025D00040F4C77081E001C0880FCA95EAF70E94F5
:1025E0002C03183028F581E09D2F977001C0880FCB
:1025F0009A95EAF70E942503802F0E941C03183049
:10260000F0F4D77081E001C0880FDA95EAF70AC0CC
:1026100080E28C0F883098F4C77081E001C0880F89
:10262000CA95EAF7DF91CF911F910F910C942C037B
:10263000802FDF91CF911F910F910C941C03DF919C
:10264000CF911F910F9108950F939C01CB01243FCF
:102650004CE5340731F188F4293DFCE53F07D9F01A
:102660002A3D4CE5340779F1283D3C45A9F506E2C1
:1026700021EE41EE68ED7CE52BC0263FFCE53F07EF
:10268000E1F0A8F0273F3C4539F507E225EE46EE9C
:1026900067EF7CE51DC007E225EE45EE69ED7CE5C0
:1026A00017C006E221EE40EE64EF7CE511C007E2C0
:1026B00025EE44EE65EF7CE50BC006E221EE42EE2E
:1026C00066EF7CE505C008E221E045EE6AED7CE5B9
:1026D0000E94B11280E008C0FC018281882319F0B9
:1026E0001092F10101C081E00F91089590932B01A8
:1026F00080932A0108959093F7018093F60108953D
:10270000E091F601F091F701309721F00190F0810E
:10271000E02D099480E00895E091F601F091F70131
:10272000309721F00280F381E02D099408952091E3
:10273000F4013091F5012817390771F09093F501F4
:102740008093F401E091F601F091F701309721F0C8
:102750000680F781E02D099408952091F2013091CF
:10276000F3012817390771F09093F3018093F20178
:10277000E091F601F091F701309721F00084F185A6
:10278000E02D09940895FC01329697E080E0915085
:1027900029F021912223D9F38F5FF9CF0895662381
:1027A00049F0FC01329608962191621729F0E8174A
:1027B000F907D1F780E0089581E008959C01FC01BC
:1027C00032969FEF80E04191461789F09F3F19F4C0
:1027D000411101C0982F8F5F8630A9F79F3F39F0D4
:1027E000F901E90FF11D97FDFA95628308950895A7
:1027F0009C012A5F3F4FFC014281461301C01282B7
:10280000019682179307B9F708950C94DE130C9480
:10281000F813029626E0FC0111922A95E9F7089533
:1028200008950C94101483E08093F8010C94111413
:10283000811102C081E001C082E08093F8010C9414
:1028400011140C94181481E08093F8010C94111465
:102850000C94231408950C942A140C942B140C94A7
:102860002A140C942A140C942A14CF930E94311425
:102870000E948F100E942F14C0E08C2F0E94AA0F7C
:10288000892B29F4CF5FC830C1F780E001C081E017
:10289000CF91089508951F920F920FB60F921124B1
:1028A0008F939F93AF93BF938091F901811113C0D0
:1028B0008091260290912702A0912802B0912902CE
:1028C0004196A11DB11D8093260290932702A093EB
:1028D0002802B0932902BF91AF919F918F910F90E1
:1028E0000FBE0F901F90189580912E02843031F109
:1028F0000E942D021092F90120E488E190E00FB6C9
:10290000F894A895809360000FBE2093600083B771
:10291000817F846083BF83B7816083BF789488950B
:1029200083B78E7F83BF0FB6F894A895809160001F
:10293000886180936000109260000FBE08950E942D
:1029400093050C94310282E084BD93E095BD9AEF2B
:1029500097BD80936E0008952FB7F894809126025A
:1029600090912702A0912802B09129022FBF0895CB
:102970002FB7F89460912602709127028091280267
:10298000909129022FBF08959C014FB7F894809130
:10299000260290912702A0912802B09129024FBFF0
:1029A000821B930B089578941F920F920FB60F928B
:1029B00011248F939F93AF93BF93809126029091A0
:1029C0002702A0912802B09129020196A11DB11DF4
:1029D0008093260290932702A0932802B0932902A5
:1029E000BF91AF919F918F910F900FBE0F901F904D
:1029F0001895F89481E08093E00080E28093D800FD
:102A0000E9ECF0E010828FE19EE40197F1F700C05D
:102A100000001DBA109268001CBC10BE1FBA1092B4
:102A20007A0010926E0010926F0010927000109257
:102A3000710010821092BC0011B814B817B81AB8FF
:102A40001DB810BA12B815B818B81BB81EB811BA0C
:102A50000C9400FE0895809102020895089508954F
:102A6000CF93DF9321E02093E9002FEF3091E8002E
:102A7000215035FD06C035ED3A95F1F700002111E2
:102A8000F5CF2091E80025FF14C0EC0140E050E0B4
:102A900068E070E00E94F0168091E8008E778093E5
:102AA000E80088E0FE01AAEFB1E001900D928A955E
:102AB000E1F7DF91CF9108950895089580912D0257
:102AC000811109C00E947D180E94DF188091E200E8
:102AD00084608093E200089510922D0208950C9472
:102AE000281460912A0281E0611101C080E00C94F9
:102AF000131490912E0281E0943009F080E06091EF
:102B00002A020C94181442E061EC81E00E94F6174E
:102B100090912E0281E0943009F080E060912A02C9
:102B20000C94211480913002833009F45FC030F49A
:102B3000813071F0823009F498C008958A3009F428
:102B400084C08B3009F46AC0893009F0A6C020C067
:102B500080912F02813A09F0A0C08091E800877F20
:102B60008093E8008091330290913402892B21F404
:102B700068E08AEF91E003C060E080E090E070E000
:102B80000E943B178091E8008B778093E8000895BE
:102B900080912F02813209F080C0809133029091A0
:102BA0003402892B09F079C08091E800877F8093F7
:102BB000E8008091E80082FD05C080912E0281111D
:102BC000F8CF6BC08091F2009091F300029731F43E
:102BD0008091F100813011F0863021F48091F10074
:102BE000809302028091E8008B7753C080912F027E
:102BF000813A09F052C08091330290913402892BBE
:102C000009F04BC08091E800877F8093E8008091B5
:102C1000E80080FFFCCF8091100136C080912F0228
:102C20008132D9F58091330290913402892BA9F534
:102C30008091E800877F8093E8000E942B188091A4
:102C40003102809310010C94930580912F02813200
:102C500021F58091E800877F8093E8000E942B187F
:102C60008091320280930302089580912F02813A6D
:102C7000A1F48091E800877F8093E8008091E800CC
:102C800080FFFCCF809103028093F1008091E800E7
:102C90008E778093E8000C942B18089584B7877F73
:102CA00084BF0FB6F894A8958091600088618093E6
:102CB0006000109260000FBE90E080E80FB6F894BC
:102CC00080936100909361000FBE0C9423140E94C6
:102CD0007D180E94DF18E2EEF0E08081846080833E
:102CE00078940C947A1B84E091E00C947B1380918F
:102CF0002E028530A9F480912E02853079F40E944D
:102D0000741480912C028823B1F30E943514882317
:102D100091F30E94DA160E949305EDCF0C949F1454
:102D2000089508950C949416292F332723303105E4
:102D3000C1F058F42130310579F02230310591F598
:102D400082E290E024E032E031C021323105E1F04E
:102D50002232310501F126C082E190E026E232E024
:102D600025C099278130910549F028F00297D1F4C8
:102D7000E4ECF1E005C0E0E0F2E002C0EEEEF1E0EC
:102D8000849190E09F0112C0672B61F489E090E08C
:102D900026E132E00BC0672B29F480E490E028E3C1
:102DA00032E004C080E090E020E030E0FA013183BE
:102DB0002083089584E189BD86E189BD09B400FEC0
:102DC000FDCF8091D8008F7D8093D8008091E00066
:102DD00082608093E0008091E00081FDFCCF089547
:102DE000CF92DF92EF92FF920F931F93CF93DF93D7
:102DF000EC018B017A010E944A18811133C0E11461
:102E0000F10439F0F70180819181081B190BC80F7B
:102E1000D91FC12CD12C0115110519F18091E800A1
:102E200085FD16C08091E8008E778093E800E1145C
:102E3000F10449F0F70180819181C80ED91ED18239
:102E4000C08285E00FC00E944A18882321F30AC07F
:102E500089918093F10001501109FFEFCF1ADF0A29
:102E6000DACF80E0DF91CF911F910F91FF90EF902B
:102E7000DF90CF90089520913502309136022617C9
:102E8000370748F06115710539F42091E8002E7775
:102E90002093E80001C0B901FC0120E06115710533
:102EA00069F180912E028823E1F18530E1F1809172
:102EB000E80083FD3AC08091E80082FD2CC080913B
:102EC000E80080FFEBCF8091F2009091F300611554
:102ED000710551F08830910538F421912093F1006B
:102EE000615071090196F3CF21E0089709F020E0C5
:102EF0008091E8008E778093E800D0CF2111D1CF68
:102F00000AC080912E02882361F0853061F08091A3
:102F1000E80083FD0AC08091E80082FFF2CF80E0E4
:102F2000089582E0089583E0089581E00895209156
:102F30003502309136022617370748F061157105C2
:102F400039F42091E8002E772093E80001C0B90100
:102F5000FC0120E06115710581F180912E0288232A
:102F600009F43EC0853009F43DC08091E80083FD3E
:102F70003BC08091E80082FD2DC08091E80080FF79
:102F8000E9CF8091F2009091F3006115710559F03D
:102F90008830910540F424912093F10031966150DE
:102FA00071090196F2CF21E0089709F020E08091A5
:102FB000E8008E778093E800CDCF2111CECF0AC0F4
:102FC00080912E02882361F0853061F08091E800C5
:102FD00083FD0AC08091E80082FFF2CF80E008956F
:102FE00082E0089583E0089581E00895982F973056
:102FF00068F59093E900981739F07091EC002091F2
:10300000ED005091F00003C0242F762F50E021FDF9
:1030100002C09F5FECCF3091EB003E7F3093EB001E
:103020003091ED003D7F3093ED003091EB00316049
:103030003093EB007093EC002093ED005093F00080
:103040002091EE0027FDE5CF80E008958F708093FA
:10305000E90081E0089580912F0287FF11C08091DF
:10306000E80082FD05C080912E028111F8CF11C0C9
:103070008091E8008B770BC080912E02882349F065
:103080008091E80080FFF8CF8091E8008E778093F0
:10309000E80008952091E4003091E50095E6409124
:1030A000EC00842F817040FF23C08091E80080FDF8
:1030B0001DC080912E02882399F0853099F080916F
:1030C000EB0085FD11C04091E4005091E50024170C
:1030D000350729F3915011F09A01E1CF84E008956A
:1030E00082E0089583E0089581E0089580E00895E6
:1030F0004091E80042FFDDCF08950E94EE180E9443
:10310000F618E0EEF0E0808181608083E8EDF0E089
:1031100080818F77808319BCA7EDB0E08C918E7F82
:103120008C9380818F7E808310922D0208950F935F
:103130001F93CF93DF930E94EE180E94F618C8EDFC
:10314000D0E088818F7788838881806888838881B0
:103150008F7D8883E7EDF0E080818068808319BCF3
:1031600010922E0210922A0210922C0210922B0220
:1031700000EE10E0F80180818B7F80838881816080
:10318000888342E060E080E00E94F617E1EEF0E024
:1031900080818E7F8083E2EEF0E080818160808399
:1031A000808188608083F80180818E7F8083888120
:1031B00080618883DF91CF911F910F910895E8ED91
:1031C000F0E080818F7E8083E7EDF0E08081816098
:1031D000808381E080932D020C949718E8EDF0E055
:1031E00080818C7F80831092E20008951092DA0033
:1031F0001092E10008951F920F920FB60F921124C2
:103200000BB60F922F933F934F935F936F937F93E0
:103210008F939F93AF93BF93EF93FF938091E100C0
:1032200082FF0BC08091E20082FF07C08091E10025
:103230008B7F8093E1000E94791B8091DA0080FFF0
:103240001FC08091D80080FF1BC08091DA008E7F64
:103250008093DA008091D90080FF0DC084E189BDA0
:1032600086E189BD09B400FEFDCF81E080932E0286
:103270000E945E1505C019BC10922E020E946C15AA
:103280008091E10080FF19C08091E20080FF15C0AD
:103290008091E2008E7F8093E2008091E200806165
:1032A0008093E2008091D80080628093D80019BC9E
:1032B00085E080932E020E9471158091E10084FFC9
:1032C00030C08091E20084FF2CC084E189BD86E19A
:1032D00089BD09B400FEFDCF8091D8008F7D809319
:1032E000D8008091E1008F7E8093E1008091E20020
:1032F0008F7E8093E2008091E20081608093E20003
:1033000080912A02882311F084E007C08091E300B5
:1033100087FD02C081E001C083E080932E020E94FD
:1033200079158091E10083FF29C08091E20083FF3D
:1033300025C08091E100877F8093E10082E0809347
:103340002E0210922A028091E1008E7F8093E1008C
:103350008091E2008E7F8093E2008091E2008061A4
:103360008093E20042E060E080E00E94F6178091E6
:10337000F00088608093F0000E946F15FF91EF913C
:10338000BF91AF919F918F917F916F915F914F917D
:103390003F912F910F900BBE0F900FBE0F901F907B
:1033A00018951F920F920FB60F9211240BB60F9221
:1033B0002F933F934F935F936F937F938F939F933D
:1033C000AF93BF93CF93DF93EF93FF93C091E90047
:1033D000CF708091EC00D82FD17080FDD0E8109292
:1033E000E9008091F000877F8093F00078940E943C
:1033F000191A1092E9008091F00088608093F00023
:10340000CD2BCF70C093E900FF91EF91DF91CF9169
:10341000BF91AF919F918F917F916F915F914F91EC
:103420003F912F910F900BBE0F900FBE0F901F90EA
:1034300018951F93CF93DF93CDB7DEB7AA970FB63A
:10344000F894DEBF0FBECDBFEFE2F2E08091F10055
:10345000819322E0E733F207C9F70E949215809129
:10346000E80083FF2EC180912F0290913002492FF6
:1034700050E04A30510508F024C1FA01E85AFF4FE4
:103480000C94951B803821F0823809F01AC108C0CD
:1034900080912B0290912C02992389F082600FC0B9
:1034A000809133028F70873008F00BC18093E90060
:1034B0008091EB0085FB882780F91092E9009091BC
:1034C000E800977F9093E8008093F1001092F1005C
:1034D000D1C0282F2D7F09F0F4C0882319F0823045
:1034E00061F0EFC080913102813009F0EAC0933081
:1034F00009F080E080932C022EC08091310281116E
:103500002AC0809133028F702FEF280F263008F0E9
:10351000D8C08093E9002091EB0020FF1CC09330BD
:1035200021F48091EB00806214C09091EB009061D7
:103530009093EB0021E030E0A90102C0440F551F39
:103540008A95E2F74093EA001092EA008091EB003E
:1035500088608093EB001092E9008091E800877FFB
:103560008093E8000E942B18ACC08111AAC0109172
:1035700031021F778091E3008078812B8093E300F4
:103580008091E800877F8093E8000E942B1880914B
:10359000E80080FFFCCF8091E30080688093E30027
:1035A000111102C082E001C083E080932E0289C025
:1035B0008058823008F085C08091310290913202AB
:1035C0008C3D53E0950779F583E08A838AE289830D
:1035D0004FB7F894DE01139620E03EE051E2E32F6E
:1035E000F0E050935700E49120FF03C0E295EF70A4
:1035F0003F5FEF708E2F90E0EA3010F0C79601C069
:10360000C0968D939D932F5F243149F74FBF8091D2
:10361000E800877F8093E8006AE270E0CE010196BF
:103620000E943B1716C06091330270913402AE01C4
:103630004F5F5F4F0E949216BC01892B09F441C075
:103640009091E800977F9093E80089819A810E9489
:1036500097178091E8008B778093E80032C080381C
:1036600081F58091E800877F8093E80080912A02AD
:103670008093F1008091E8008E7772CF811121C094
:10368000809131029091320299270297D4F480916F
:10369000E800877F8093E8008091310280932A02BE
:1036A0000E942B1880912A02811106C08091E300AC
:1036B00087FD02C081E001C084E080932E020E9459
:1036C00083158091E80083FF0AC08091E800877F1E
:1036D0008093E8008091EB0080628093EB00AA96D3
:1036E0000FB6F894DEBF0FBECDBFDF91CF911F9113
:1036F00008950895CF9380912E028823A1F0C09160
:10370000E900CF709091EC00892F817090FD80E8E6
:10371000C82B1092E9008091E80083FD0E94191ADD
:10372000CF70C093E900CF910895EE0FFF1F0024E2
:10373000001C0BBE0790F691E02D0994FB01DC0103
:1037400004C08D910190801921F441505040C8F778
:10375000881B990B0895F999FECF92BD81BDF89A07
:10376000992780B50895A8E1B0E042E050E00C94BC
:10377000DF1B262FF999FECF92BD81BDF89A0197E4
:1037800000B4021639F01FBA20BD0FB6F894FA9AA9
:10379000F99A0FBE08950396272F0E94BA1B0E9424
:1037A000B91B252F0E94BA1B242F0C94BA1B01961B
:1037B000272F0E94BA1B0C94B91BDC01CB01FC0122
:1037C000F999FECF06C0F2BDE1BDF89A319600B47A
:0E37D0000D9241505040B8F70895F894FFCF85
:1037DE00C800C8012B1530155C155D152E152F155B
:1037EE00016766656463626160C1C0979695949344
:0A37FE0092F7F6F5F4F3F2F1F00093
:00000001FF
